:10079B005452414E5A004241554400525F5348490E
:1007AB00465400494E565F52454300494E565F54DE
:1007BB0052414E530000C8CCDF73696E7573625F94
:1007CB0073747265616D2E62696E00312E3000C4D8
:1007DB00C0D2C030362F32322F30390031343A3557
:1007EB00353A343600FF079BFF07A1FF07A6FF072B
:0707FB00AEFF07B6FF07C0C7
:03002A00011200C0
:10000300C2AFC28E53890F438910758BE0758DC1C2
:07001300D2ABD28ED2AF2266
:1008EB00E4F515C2CAD2CDD2CCC2C9E513F5CBE51E
:1008FB0014F5CA85CBCD85CACC75B710D2CAC299AF
:09090B00C298D29CC2B2D2B12202
:03001B000208A632
:1008A600C0E0C0D0C28E758BE0758DC1200A06757A
:1008B600A61E75A6E10512D204E51560020515050A
:1008C60017E517540F7017D211E517543F7002D26F
:1008D60000E516D394644004D20A80020516D28E2F
:0508E600D0D0D0E0328B
:10071B00C207C2067513FF7514B2C296C2971208B0
:10072B005A120222E4F50AF50FF50BF510C20A1264
:10073B00000375A70775A61E75A6E11208EB120834
:10074B000212001EE4900108F0E4F516A20692973F
:10075B00309822C29874082510F582E43400F58392
:10076B00E599F00510900108E004F0D206E0D3946F
:10077B00084002D2B2309902C299900108E0C394AA
:10078B00045002C2B230B2C12006BED20680BA22D9
:10022200E4F523E52375F003A424F0F582E4340712
:10023200F583E493FB740193FA740293F912003686
:1002420070030203D4E4F525F526F5247409252468
:10025200F582E43401F583E070030203CFE52375F0
:10026200F003A424F0F582E43407F583E493FB74ED
:100272000193FA740293F985258275830012004F67
:10028200FF74092524F582E43401F583E0B50708FB
:1002920075260105250203CAE52670030203CAE595
:1002A2002375F003A424F0F582E43407F583E49384
:1002B200FB740193FA740293F98525827583001207
:1002C200004F60030203C5E52314605C147003024F
:1002D20003B91470030203BD1470030203C12404A2
:1002E20060030203CF74092524F9E43401FA7B0187
:1002F200C0031B8B2E752F00753000E4F531D0033F
:100302001203D58F2A8E298D288C27AB2AAA29A9D8
:1003120028A8277FB07E717D0B7C001200B81201E5
:100322004A8E138F140203CF74092524F9E4340191
:10033200FA7B01C0031B8B2E752F00753000E4F58C
:1003420031D0031203D58F2A8E298D288C27E4FF02
:10035200FEFDFCAB2AAA29A928A827C312015860CE
:100362001FAB2AAA29A928A827E47F847E1EFDFCA8
:100372001200B812014A9001CDEFF0E49001CCF0E6
:10038200E47FB07E04FDFCAB2AAA29A928A827D3C2
:1003920012015840389001CC7401F0AB2AAA29A965
:1003A20028A8277F487EE8FD7C001200B812014A87
:1003B2009001CDEFF08016D2078012D20D800ED2BE
:1003C20009800AE4F526F525052402024E052302DA
:0203D200022502
:0103D4002206
:10080200C2A94389029001CDE0F58CE0F58A75D941
:100812000475DC4975DD4975DA31E4F5E9F5F9F578
:10082200EBF5FB9001CCE0601675EC1075ED10E471
:10083200F5FCF5FD750E08750C10750D018013752C
:10084200EC8075ED80E4F5FCF5FD750E80F50C7518
:080852000D10E4F5EAF5FA22AD
:0B001E00E4FFD28C75D840D2AEF51183
:0100290022B4
:030033000205794A
:10057900C0E0C083C082C0D030D82FC3E5EC95EA73
:10058900C3950E5012E50D25ECF5EC30D70405FCAA
:10059900801685FCFC8011C3E5EC950DF5EC30D790
:1005A9000415FC800385FCFCC2D830D902C2D930BD
:1005B900DA54E50C700405FC8010E50C25ECF5EC2B
:1005C90030D70405FC800385FCFC300715E508C31A
:1005D90013F5083093042480F508200D166308806C
:1005E9008011E50825E0F5083093020508200D0380
:1005F900630801A2939296050FE50F5407700585CC
:100609000899F508C2DA30DB74C2DBE50C70040521
:10061900FD8010E50C25EDF5ED30D70405FD8003CF
:1006290085FDFD20060B300904D2928050C29280CC
:100639004C30070DE509139292E509C313F50980BA
:100649000BE509339292E50925E0F5090511E51154
:1006590054077029900108E0D39400401E050B74DB
:1006690008250BF582E43400F583E0F50920090338
:100679006309FF900108E014F08002C206D0D0D0CF
:0606890082D083D0E032B4
:10091400E5D220E0FBC2AF438E2075D2028F8275F0
:0C0924008300E0FFE4F5D2538EDFD2AF79
:0109300022A4
:10093100E5D220E0FBC2AF43D2028F82758300ED86
:0A094100F075D25063D250D2AF22FD
:10085A00E4FEEEC39480503EEE247FFF1209147426
:10086A00092EF582E43401F583EFF074092EF5823E
:10087A00E43401F583E0701B74092EF582E4340137
:10088A00F5837420F0740A2EF582E43401F583E4CA
:0B089A00F080030E80BCE4900188F0A9
:0108A5002230
:0300000002068F66
:0C068F0078FFE4F6D8FD75813C0206D629
:10069B0002071BE493A3F8E493A34003F68001F253
:1006AB0008DFF48029E493A3F85407240CC8C33360
:1006BB00C4540F4420C8834004F456800146F6DF2F
:1006CB00E4800B010204081020408090002AE47E95
:1006DB00019360BCA3FF543F30E509541FFEE49324
:1006EB00A360010ECF54C025E060A840B8E493A3EB
:1006FB00FAE493A3F8E493A3C8C582C8CAC583CA16
:10070B00F0A3C8C582C8CAC583CADFE9DEE780BECD
:01002D0000D2
:10003600BB010689828A83E0225002E722BBFE02C8
:09004600E32289828A83E49322FB
:10004F00BB010CE58229F582E5833AF583E0225066
:10005F0006E92582F8E622BBFE06E92582F8E222B0
:0D006F00E58229F582E5833AF583E49322CA
:10007C0075F008758200EF2FFFEE33FECD33CDCC3B
:10008C0033CCC58233C5829BED9AEC99E5829840BE
:10009C000CF582EE9BFEED9AFDEC99FC0FD5F0D69B
:1000AC00E4CEFBE4CDFAE4CCF9A88222B800C1B9C5
:1000BC000059BA002DEC8BF084CFCECDFCE5F0CB03
:1000CC00F97818EF2FFFEE33FEED33FDEC33FCEB3C
:1000DC0033FB10D703994004EB99FB0FD8E5E4F9F7
:1000EC00FA227818EF2FFFEE33FEED33FDEC33FCE4
:1000FC00C933C910D7059BE99A4007EC9BFCE99AD8
:10010C00F90FD8E0E4C9FAE4CCFB2275F010EF2F1C
:10011C00FFEE33FEED33FDCC33CCC833C810D7071C
:10012C009BEC9AE899400AED9BFDEC9AFCE899F857
:0E013C000FD5F0DAE4CDFBE4CCFAE4C8F922EA
:0E014A00C3E49FFFE49EFEE49DFDE49CFC22C6
:10015800EB9FF5F0EA9E42F0E99D42F0E89C45F0FD
:010168002274
:1003D5008B2B8A2C892DE4F537F536F535F534F573
:1003E50032F533E52F4530452E6012EBC0E0EAC00B
:1003F500E0E9C0E0AB2EAA2FA9301201B8AB2B055E
:100405002DE52DAA2C7002052C14F9120036F538AD
:10041500C394094007E538D3940D40E1E5386420DD
:1004250060DBE538B42D054333038016E538B42B7E
:1004350005433301800C74FF252DF52D74FF352CF4
:10044500F52CE53160046410703FAB2BAA2CA92D67
:1004550012003664306009E531702E75310A802945
:1004650090000112004FFF64786004EFB458134305
:1004750033017531107402252DF52DE4352CF52C3D
:100485008007E5317003753108AB2B052DE52DAAE5
:100495002C7002052C14F9120036F538C39461400E
:1004A5000AE538D3947A50035338DF74D02538F5EC
:1004B50038C3940A400CE5389411406D74F9253819
:1004C500F538E538D39531506043330185373C85A0
:1004D500363B85353A853439AF317E00E4FCFDABDA
:1004E50037AA36A935A834120169C8ECC8C9EDC9BF
:1004F500CAEECACBEFCBE4FCFDFEEB2538F537EEB3
:100505003AF536ED39F535EC38F534AF37AE36AD6D
:1005150035FCAB3CAA3BA93AA839D3120158500384
:1005250002048E43330402048EE53320E003E480A5
:100535002DE52F4530452E601EAB2BE52D24FFF90B
:10054500E52C34FFFAEBC0E0EAC0E0E9C0E0AB2EF1
:10055500AA2FA9301201B8E53330E20774FFFFFE78
:10056500FDFC22E533AF37AE36AD35AC3430E103B3
:0405750002014A2213
:10016900E88FF0A4CC8BF0A42CFCE98EF0A42CFC35
:100179008AF0EDA42CFCEA8EF0A4CDA8F08BF0A4B3
:100189002DCC3825F0FDE98FF0A42CCD35F0FCEB12
:100199008EF0A4FEA9F0EB8FF0A4CFC5F02ECD39D7
:0F01A900FEE43CFCEAA42DCE35F0FDE43CFC2244
:1001B800BB011A89828A83D0F0D0E0F8D0E0F9D068
:1001C800E0FAD0E0FBE8C0E0C0F00202105016E907
:1001D800F8D083D082D0E0F9D0E0FAD0E0FBC0823A
:1001E800C083020207BBFE16E9F8D083D082D0E0B4
:0F01F800F9D0E0FAD0E0FBC082C08302021922E6
:09020700EBF608EAF608E9F6221C
:09021000EBF0A3EAF0A3E9F022EF
:09021900EBF208EAF208E9F22216
:00000001FF
